:020000040000FA
:10000000831670308F001028AB000308AC000A087C
:10001000AD002D088A002C088300AB0E2B0E0900C2
:10002000FB3085007F308100DC30860003309B0090
:1000300040309F00F9309200831240309F003C30E6
:10004000970083162430980018309900831290305E
:1000500098007D30950007309200FD20A001A2019C
:10006000A4018C1A402841302002031D3E28B520EF
:100070002608F720043085062708F720C8203128F5
:100080001819A9289818AE281A08A0004130200293
:100090000319312842302002031D50280511312850
:1000A00043302002031D5B282208F7202408F72094
:1000B0004230A000312844302002031D31280515AC
:1000C000831790308400B52084132608800084179D
:1000D00027088000840A0408F03C031D6328A03030
:1000E0008400B520831326088000840A2708800036
:1000F000840A0408003C031D712883179030840093
:1001000084130008F72084170008F720840A0408E5
:10011000F03C031D80288313A03084000008F720E2
:10012000840A0008F720840A0408003C031D9D2867
:100130000921D130F72009215B288C1E8E281A084E
:10014000A00042302002031D8E2805114230A0007D
:1001500031281A08FD20FD20981C31281A08181291
:100160001816FD20FD20FD20312849309F00132165
:100170001F151F19B9281E0C7F39A60041309F009A
:1001800013211F151F19C2281E0C7F39A700080054
:100190000608A100C030A11FD728211FD628211E84
:1001A000D528A11DD428013E013E013E013E013E5D
:1001B000A50024020319DF282508A400F72005085C
:1001C000A100B030A11FEE28211FED28211EEC2830
:1001D000A11DEB28013E013E013E013E013EA30070
:1001E0002202031908002308A200F7200800831642
:1001F000981CF82883129900080005156430042122
:100200000511643004210800AA000921AA0B052960
:100210000800F130A900132113210000A90B0B29BC
:100220000000000008000830A8000000A80B1529F5
:06023000000000000800C0
:02400E00303F41
:02401000FC3F73
:00000001FF
